:02000000502A84
:080008002028820700340134B6
:10001000013400340134003400340134013400343C
:1000200000340134003401340134003482072034B8
:100030003234313420348207203430343034353493
:10004000BB000308BC000408BD000B1E36288B1C37
:1000500036281430840004308618E0303F22031C18
:1000600034281915031919110B122C2A0B1DD62926
:10007000B23081000B1106081039950003109E0C58
:100080002030151A9E049F0B4C281E0840389D00F6
:10009000961406309F009E01FF301507A40DA30D96
:1000A000A20DA10DA00D971C5728AC0BA9291E303D
:1000B000AC002708AB002608AA002508A9002308E1
:1000C000A7002208A6002108A500201C6A28A7096D
:1000D000A609A509A801A018A80A250E0E39052011
:1000E000A80625080C390520A806260E0739052084
:1000F000A80626080C390520A806270E0D3905206C
:10010000A806270802390520A80603198A28A41F73
:1001100055298C28A41B5529A8012018A80A250EAA
:1001200007390520A806250806390520A806260E49
:1001300003390520A80626080E390520A806270E33
:1001400006390520A806270809390520A80603193D
:10015000AC28241F5529AE28241B5529A801A01816
:10016000A80A250E0B390520A80625080B390520FD
:10017000A806260E01390520A80626080F390520F5
:10018000A806270E03390520A806270804390520EC
:10019000A8060319CE28A41E5529D028A41A55292B
:1001A000A8012018A80A250E05390520A80625084B
:1001B0000D390520A806260E08390520A8062608B0
:1001C0000F390520A806270E09390520A80627089B
:1001D0000A390520A8060319F028241E5529F228FB
:1001E000241A5529A8012018A80A250E0A39052025
:1001F000A80625080E390520A806260E0C3905206C
:10020000A806260807390520A806270E0C39052060
:10021000A80627080D390520A80603191229A41DD0
:1002200055291429A4195529A801A018A80A250E92
:1002300002390520A80625080D390520A806260E36
:100240000E390520A80626080A390520A806270E1B
:1002500002390520A806270807390520A806031932
:100260003429241D55293629241955292408230405
:1002700022042104031955292408230522052105F8
:10028000FF3A031955291917971C4D29123084007C
:1002900010303F22031819166029971480309200FD
:1002A000930019129912B01760291913971C60292D
:1002B00012308400C0303F22031C602997104E2961
:1002C000191EA929AF0A171D88292F082E06031DFC
:1002D000A929AD0A66302906031D762926082D06B0
:1002E0000739031D762916174030792916138830EF
:1002F000B017133084003F22031C90290319822970
:10030000991690299912171180309300B017A929D6
:1003100066302906031DA92980309300B0171715F0
:10032000AF0126080739AD002708AE00AE0CAE0CB1
:100330002E0C1F39023EAE00B017991EA929191FB5
:10034000A929161FA9292B08B1002A080339B000D2
:10035000A929161DBA298316860183128511051154
:10036000971905151A0886008515851183168609C3
:1003700083121611961CD62909309C000514C02939
:10038000C12900001B08B700B70BC4299C0BC92961
:10039000D1299D0C0318CF2905140000C22905108E
:1003A000C229D22900009610D52905100B1C292A34
:1003B0000608103915060319152A16100F30840087
:1003C0000108263EB700031CF5290319052AF83E4B
:1003D000031CF0293708F03E031816140730B70045
:1003E0003708991901308102052AB709B70A370879
:1003F000F83E031C012A3708F03E03181614073094
:10040000B700370899190130810701301618F93003
:100410003F22031C152A031D142A9911100B112ABF
:1004200003309000E922152A99152930861F1A2ACF
:100430003A221D2A061F292A3422D122161606081E
:10044000C039031D1F2A04301A230608C039031DB2
:100450001F2A8B150B100B163D088400BB0E3C08A1
:1004600083003B0E8B1009008E038E1F080028307E
:100470008E0008008E0A0E0203198E000800B700D5
:100480008007B71F482A03184E2A8001031408006A
:10049000031C4E2A80018009031408000310080081
:1004A00014301A2387228B17402380239823161E8B
:1004B0005B2A802316129910061D99141910861DA7
:1004C0001914190818060319742A19089800C93054
:1004D00036230730B800980C2B30031C58303A23D1
:1004E000B80B6B2A190898008B133008B500310837
:1004F000B6008B1735083206031D812A36083306ED
:10050000031D8C2311081006031D9823572A8316F8
:10051000860186098501051583121E3005194130B3
:100520009B008316850183120510851005160A307D
:100530001A23A030BE220512000005163F30BE224D
:10054000A030BE224F30BE22A030BE220512F822BB
:10055000D12206309F009E019601B1220B108B150F
:100560000800803094008F0092009300940099015D
:100570009801B0170330900099110800B7000830B7
:10058000BA008510831686108312B70D86100318E3
:10059000861485148510BA0BC52A83168614831217
:1005A000080001308C0097308D000E088D0703186D
:1005B0008C0A05120C08BE220D08BE220330BE2292
:1005C000E830BE22051605120023B1220330E922CD
:1005D00008008B12900080308F009911100883164C
:1005E000C43E81008312B23081000B118B160800CB
:1005F0002830890083160814831208088E0008002A
:100600000E0888002830890083168818052B0815E5
:1006100055308900AA308900881483120800E93017
:10062000013E031C102B08006430B9000F23B90BE6
:10063000162B0800BA001423BA0B1B2B080001303C
:10064000B400B60DB50DB40D03182F2B0330B5074C
:10065000B51DB5023030B507B51FB502212B3408E2
:100660003823350E382335083823080097113B2BE3
:100670000F39303E97159A00161516193D2B0800B4
:1006800038303623142338303623383036231423B9
:1006900038303623063036230C30362301303623EB
:1006A0001423833036236B303A2386303623493087
:1006B0003A2344303A238930362353303A234930A1
:1006C0003A2343303A2342303A2357303A234630D4
:1006D0003A2350303A23C230362330303A23623046
:1006E0003A2373230800C53036230330B8002D3079
:1006F0003A23B80B782B20303A23B217B0170800F2
:100700000130B5000E081D3EB6000318B50A1612DA
:10071000803036231F2308003508B2003608B300A6
:10072000B51F942B73230800C53036231F23080000
:1007300010089100C0303623110816203A23110802
:060740001B203A23080013
:02400E00F93F78
:10420000560065007200200031002E0030002000B2
:1042100044004700500053002E00410053004D0061
:1042200063006F0070007900720069006700680029
:10423000740020004A0069006D00200042006900FF
:104240007800620079002000310039003900380020
:044250001100000059
:00000001FF
